:100000000C94EB030C9432040C94A9070C94320466
:100010000C9432040C9432040C9432040C94320488
:100020000C9432040C9432040C9432040C945E0D43
:100030000C9432040C948B1B0C9432040C943204F8
:100040000C9432040C9432040C9432040C94D51B9E
:100050000C9432040C9432040C9432040C94320448
:100060000C9432040C9432040C9432040C94320438
:100070000C9432046005B3059505D705EB05F10531
:10008000F505F905FD050106050608060C0610062E
:10009000310E530E410F530E410F980EBB0E410F00
:1000A000100F230F1B121B1248124812A312BF1469
:1000B000BF14BF14DF12BF14DA13DA139514BF1480
:1000C000BF14AB148042803E3C3A3B456843413FFD
:1000D0003D2B3567697A790078141E806A801D1679
:1000E000041A1F806B061B07082120806C2C19093D
:1000F000171522806D11050B0A1C23806E80100DD0
:10010000182425806F360E0C122726807037380F82
:1001100033132D80717534802F2E8072397D2830F5
:10012000803180738064808076802A778059745C07
:100130005F66808062635A5D5E60295344575B56F8
:100140005561478080808040808080808080808072
:1001500080808080807E80807C80808080808080A5
:100160008080807B800180038080807F8080808091
:100170008080806580800280808080808080808018
:10018000808080808080808080808080808054809B
:100190008080808080808080808080808080588087
:1001A000808080808080808080808080804D8050B2
:1001B0004A808080494C51804F52808080804E80A0
:1001C000464B48800A0025303862003A200025302E
:1001D0003258000A722F63203031323334353637CB
:1001E0000A00756E65787065637465642073636179
:1001F0006E20636F64652061742045305F46303A3D
:1002000020253032580A00756E6578706563746514
:1002100064207363616E20636F646520617420469F
:10022000303A20253032580A00756E657870656363
:10023000746564207363616E20636F64652061740C
:100240002046303A20463028636C65617220616E2A
:100250006420636F6E742E290A00756E6578706570
:1002600063746564207363616E20636F64652061ED
:10027000742045303A20253032580A00756E657872
:10028000706563746564207363616E20636F646579
:1002900020617420494E49543A20253032580A00D2
:1002A0004F76657272756E0A0025690D0A007062DC
:1002B00075663A2066756C6C0A005B735D004B6571
:1002C00079626F6172642073746172742E0A0055D2
:1002D000534220636F6E666967757265642E0A000B
:1002E0005B575D005B535D005B525D003003500067
:1002F00053002F00320020006B006500790062007F
:100300006F00610072006400200063006F006E00E7
:1003100076006500720074006500720000000E0334
:1003200074002E006D002E006B002E0000000403F0
:10033000090409027400040100A03209040000014C
:10034000030101000921110100012240000705817C
:100350000308000A0904010001030000000921113B
:100360000100012236000705820308000A09040281
:1003700000020300000009211101000122220007F0
:10038000058303200001070503032000010904037E
:1003900000010300000009211101000122390007BA
:1003A0000584032000011201100100000008EDFE89
:1003B000126501000102000105010906A1010507FE
:1003C00019E029E715002501950875018102050846
:1003D0001901290595057501910295017503910192
:1003E0000507190029F71500250195F87501810207
:1003F000C00631FF0974A1010975150026FF00959B
:1004000020750881020976150026FF0095207508E1
:100410009102C005010980A101850216810026B75D
:10042000001A81002AB700751095018100C0050CE3
:100430000901A1018503160100269C021A01002A68
:100440009C02751095018100C005010906A10105F6
:100450000719E029E7150025019508750181029526
:100460000175088101050819012905950575019196
:10047000029501750391010507190029FF15002652
:10048000FF00950675088100C00A0025303258200B
:10049000006B6579626F6172645F7265706F727410
:1004A0003A20004C45443A20253032580A00646511
:1004B0006C5F6B65795F6269743A2063616E277463
:1004C0002064656C3A20253032580A006164645F0C
:1004D0006B65795F6269743A2063616E277420618D
:1004E00064643A20253032580A003F00433E200021
:1004F0004C25640A000A092D20436F6E736F6C65EA
:10050000202D0A4553432F713A09717569740A0009
:100510000A092D204D61676963202D0A643A096438
:10052000656275670A783A096465627567206D616E
:10053000747269780A6B3A096465627567206B6545
:1005400079626F6172640A6D3A0964656275672049
:100550006D6F7573650A763A0976657273696F6EA9
:100560000A733A097374617475730A633A09636FA5
:100570006E736F6C65206D6F64650A302D343A09B7
:100580006C61796572302D34284631302D4634291E
:100590000A506175733A09626F6F746C6F616465BC
:1005A000720A6E3A094E4B524F0A003F004E4B52B0
:1005B0004F3A206F66660A004E4B524F3A206F6EDC
:1005C0000A0074696D65725F72656164333228294F
:1005D0003A202530346C580A006B6579626F61727D
:1005E000645F6E6B726F3A2025580A006B65796202
:1005F0006F6172645F69646C653A2025580A006B0C
:100600006579626F6172645F70726F746F636F6C33
:100610003A2025580A00686F73745F6B6579626FC2
:100620006172645F6C65647328293A2025580A005A
:100630000A092D20537461747573202D0A004743F5
:10064000433A20342E392E32204156522D4C494205
:10065000433A20312E382E3073766E204156525F49
:10066000415243483A2061767233350A004F505464
:10067000494F4E533A204C5546412045585452411B
:100680004B455920434F4E534F4C4520434F4D4D02
:10069000414E44204E4B524F204B45594D41505FE7
:1006A00053454354494F4E20343039360A004255A1
:1006B000494C443A20323232616462372D646972A7
:1006C0007479202831313A35313A35382053657004
:1006D0002031372032303136290A005649443A2039
:1006E00030784645454428742E6D2E6B2E292050B7
:1006F00049443A203078363531322850532F322051
:100700006B6579626F61726420636F6E7665727477
:10071000657229205645523A203078303030310AFF
:1007200000444553433A20636F6E766572742050DF
:10073000532F32206B6579626F61726420746F2071
:100740005553420A000A092D2056657273696F6E6F
:10075000202D0A000A6D6F7573653A206F66660A70
:10076000000A6D6F7573653A206F6E0A000A6B653B
:1007700079626F6172643A206F66660A000A6B657F
:1007800079626F6172643A206F6E0A000A6D61745B
:100790007269783A206F66660A000A6D6174726940
:1007A000783A206F6E0A000A64656275673A206FB6
:1007B0006E0A000A64656275673A206F66660A0011
:1007C0000A0A626F6F746C6F616465722E2E2E2040
:1007D00000433E20000011241FBECFEFD4E0DEBF57
:1007E000CDBF04B603FE27C0809152029091530200
:1007F000A0915402B09155028730904BA740B04B66
:10080000D1F410925202109253021092540210929C
:10081000550214BE84B7877F84BF0FB6F894A8959D
:1008200080916000886180936000109260000FBE2C
:10083000E0E0F8E3099511E0A0E0B1E0EAE6FCE3CE
:1008400002C005900D92A432B107D9F722E0A4E2CC
:10085000B1E001C01D92A235B207E1F70E94A40ADF
:100860000C94331E0C940000FF93EF93E09124014D
:10087000F0912501309709F00995EF91FF910895C6
:10088000FC018591803011F0EFDFFBCF0895FF2749
:10089000E0E230E247FF0CC0419597FF09C0EDE26E
:1008A0006095709580959095611D711D811D911DBC
:1008B00027FF02C0219530E350E2AA27660F771F79
:1008C000881F991FAA1FA41710F0A41B63955A959F
:1008D000A9F7AA3008F0A95FA05DAF93F395611561
:1008E00071058105910541F7ED3211F4EF93F39510
:1008F000F21718F43F93F395FBCF8F91B5DFFA957C
:10090000E1F70895E991F9918591803021F08532E0
:1009100019F0AADFF9CF089520E0E89455915532F7
:10092000C1F3503311F4689455915A3348F450533D
:1009300090F3220F022E220F220F200D250FF4CF4D
:100940000EF4219589919991533619F3533729F172
:10095000533559F1BC0188279927E8945C3621F476
:100960008991999168945591543639F446EF7EF007
:1009700077FF0DC08FEF9FEF0AC055374AE039F07F
:10098000583540E121F0523642E009F00895FF93D6
:10099000EF937DDFEF91FF91B7CFFF93EF93FC01D2
:1009A00081918030B9F360DFFBCFFF93EF9368DF75
:1009B000F1CFDF93CF93CDB7DEB72596A3DFCF91ED
:1009C000DF910895E82FE695E695E695F0E0E85D7D
:1009D000FE4F4081282F277081E090E002C0880FF1
:1009E000991F2A95E2F7242F30E028233923232B5F
:1009F00029F4842B808381E0809327010895E82FD8
:100A0000E695E695E695F0E0E85DFE4F2081382F0B
:100A1000377081E090E002C0880F991F3A95E2F7A5
:100A2000422F50E048235923452B31F080958223F3
:100A3000808381E0809327010895E8E2F1E080E27D
:100A40008E0F11928E13FDCF089580913E0281602A
:100A500080933E020E94B806E8E2F1E080E28E0F49
:100A600011928E13FDCF0895CF931092270180919C
:100A7000470186FF03C08EEF0E94FF040E9491078A
:100A8000C82F882361F01F928F9389EA92E09F9389
:100A90008F930E94D9040F900F900F900F90809128
:100AA0004A018111C4C0E09126018E2F90E08E3062
:100AB000910508F0BAC0FC01E65CFF4F0C942D1EB6
:100AC000C43899F030F4CC2391F0C338C9F483E8EA
:100AD000AAC0C13E41F0C03F21F0C03E89F482E08F
:100AE0007DC081E07BC084E079C08CEF9CC00E9417
:100AF0001D050E94DC1480EA92E00E94400495C02B
:100B0000C7FD02C08C2F8FC00E941D050E94DC14FF
:100B10001F92CF938CE792E09F938F930E94D9040A
:100B20000F900F900F900F9080C0C93509F47DC0D1
:100B300020F4C23109F479C008C0CE3721F0C03F9B
:100B400021F483E04BC08BE049C0C7FD03C08C2F6C
:100B5000806869C00E941D050E94DC141F92CF931B
:100B60008AE592E0D9CFC43831F0C03F31F0C338C4
:100B700089F483E824C08CEF22C00E941D050E94E6
:100B8000DC1489E292E09F938F930E94D9040F9026
:100B90000F904DC0C7FD02C08C2F11C00E941D05D3
:100BA0000E94DC141F92CF9387E092E0B5CFC23150
:100BB000E1F1C935D1F1C7FD05C08C2F80680E94D5
:100BC000FF0433C00E941D050E94DC141F92CF93C6
:100BD00082EE91E0A1CFC43141F585E080932601FA
:100BE00026C0C73711F586E0F9CFC13EF1F487E0A2
:100BF000F5CFC03FD1F488E0F1CFC431B1F489E042
:100C0000EDCFC03F91F48AE0E9CFC73771F40AC055
:100C1000C03E59F48CE0E2CFC03F39F48DE0DECF26
:100C2000CE3719F48EEF0E94E2041092260181E083
:100C3000CF910895E82FF0E0E85DFE4F80810895A0
:100C4000CF92DF92EF92FF920F931F93CF93DF9398
:100C500083ED91E00E94400488E2E82E81E0F82EC6
:100C6000C0E0D0E09EECC92E91E0D92E06EC11E058
:100C7000DF93CF93DF92CF920E94D9048BEC91E067
:100C80000E944004F70181917F010E94241B1F9262
:100C90008F931F930F930E94D90484EC91E00E94DC
:100CA000400421968DB79EB708960FB6F8949EBF64
:100CB0000FBE8DBFC032D105D9F6DF91CF911F9104
:100CC0000F91FF90EF90DF90CF900895982F82FBC7
:100CD000882780F990FD826091FD84600C943C0827
:100CE0004FB7F89420914B0130914C0180914D0108
:100CF00090914E018217930781F0F901EE0FFF1FCB
:100D0000E15BFE4F808191812F5F3F4F2F71332731
:100D100030934C0120934B0102C080E090E04FBF24
:100D20000895CF93DF93EC010E944B08882341F094
:100D3000209731F085E08A95F1F700002197F4CFF4
:100D4000CE01DF91CF910895CF93DF93C2E3D0E03E
:100D50000E944B08811108C0209731F085E08A95E8
:100D6000F1F700002197F4CFCE01DF91CF910895E4
:100D70000E9448080E945808E9E6F0E080818860F7
:100D80008083E99A08958AE1815019F40E947006DF
:100D900008959FB7F89440914D0150914E012091D4
:100DA0004B0130914C019FBF4217530779F7EFE990
:100DB000FFE03197F1F700C00000E6CFEF92FF921D
:100DC0000F931F93CF93DF93E82E10924A01E99877
:100DD0000E9445080E9458088FE891E00197F1F7BA
:100DE00000C000000E9455080E94480880E197E278
:100DF0000E949106892B11F48AE077C0C0E0D0E010
:100E000011E0F12C01E090E59A95F1F7C7010C2E65
:100E100002C0959587950A94E2F780FF04C01027D9
:100E20000E94580802C00E9455080E94A406892BFF
:100E300011F482E05AC082E390E00E949106892B6F
:100E400011F483E052C02196C830D105E1F680E567
:100E50008A95F1F7112319F00E94580802C00E94E8
:100E600055080E94A406892B11F484E03EC082E359
:100E700090E00E949106892B11F485E036C090E540
:100E80009A95F1F70E945808C2E3D0E00E945B08EF
:100E9000882341F0209741F025E02A95F1F70000E2
:100EA0002197F4CFCD2B11F486E01FC082E390E0B0
:100EB0000E949106892B11F487E017C00E94A406B6
:100EC000892B11F488E011C0C2E3D0E00E945B08D6
:100ED000811108C0209741F085E08A95F1F7000064
:100EE0002197F4CFCD2B81F489E080934A010E94B1
:100EF00048080E945808E99A80E0DF91CF911F913D
:100F00000F91FF90EF9008950E9448080E945808A2
:100F1000E99ADF91CF911F910F91FF90EF900C9480
:100F2000C3064FB7F89420914D0130914E01809146
:100F30004B0190914C014FBF2817390729F01092AF
:100F40004A010E947006089580E280934A0180E081
:100F500008951F920F920FB60F9211242F933F9373
:100F60004F935F936F937F938F939F93AF93BF93B1
:100F7000CF93EF93FF930E944B0881116BC0809138
:100F800049018F5F809349018A3028F4823068F4E8
:100F9000813031F054C08A30D9F08B3029F14FC004
:100FA0000E945B0881114BC055C080914801869515
:100FB000809348010E945B08882309F44BC080910C
:100FC0004801806880934801809100018F5F40C094
:100FD0000E945B0890910001882319F090FF2FC0B8
:100FE00039C090FD2CC036C00E945B08882339F1BF
:100FF0004091480150E0CFB7F89480914D01909115
:101000004E019C012F5F3F4F2F71332760914B01A1
:1010100070914C012617370761F0880F991FFC016A
:10102000E15BFE4F5183408330934E0120934D018D
:1010300004C08EEA92E00E944004CFBF04C08091B9
:10104000490180934A01109249011092480181E0C0
:1010500080930001FF91EF91CF91BF91AF919F914C
:101060008F917F916F915F914F913F912F910F9051
:101070000FBE0F901F901895CF93C82F8DEE0E9432
:10108000DE068C2FCF910C94DE065998519A089564
:101090005198599A08955198599A85E08A95F1F78F
:1010A000000089B18695817008955898509A0895E6
:1010B0005098589A08955098589A85E08A95F1F773
:1010C000000089B1817008958091B201089508955A
:1010D0009FB7F894109291019FBF9091490294306C
:1010E00009F057C09091E9009F703091EC00232FD8
:1010F000217030FD20E8922B23E02093E90020911D
:10110000EB0020FF43C02091EE0027FF3FC020915D
:101110008F01222321F02091E80025FF37C0109293
:101120008F0126E03091E80035FD15C0309149026D
:10113000343061F53091EB0035FD28C0215021F4A9
:1011400081E080938F0122C0EFE9FFE03197F1F752
:1011500000C00000E7CF8093F1008091E80085FD9A
:101160000AC08091E80080FFFCCF8091E8008E7774
:101170008093E80006C08FB7F89421E02093910196
:101180008FBF9F709093E90080E008959F709093C7
:10119000E9008FEF0895CF93DF9300D01F92CDB772
:1011A000DEB720914902243021F523E029839B8377
:1011B0008A8382E08093E9008FEF9091E80081506C
:1011C00095FD06C095ED9A95F1F700008111F5CFD8
:1011D0008091E80085FF0DC040E050E063E070E0E2
:1011E000CE0101960E946A0B8091E8008E77809371
:1011F000E8000F900F900F90DF91CF910895CF935B
:10120000DF9300D01F92CDB7DEB79C0180914902D9
:10121000843019F592E099833B832A839093E90007
:101220008FEF9091E800815095FD06C095ED9A955D
:10123000F1F700008111F5CF8091E80085FF0DC026
:1012400040E050E063E070E0CE0101960E946A0B3E
:101250008091E8008E778093E8000F900F900F90B8
:10126000DF91CF910895CF93DF93EC0190914902E4
:10127000943009F046C080910B018823D9F0809109
:101280000C018823B9F09093E9008FEF9091E8006A
:10129000815095FD06C095E19A95F1F70000811106
:1012A000F5CF8091E80085FF2CC040E050E060E27F
:1012B00070E017C081E08093E9008FEF9091E80023
:1012C000815095FD06C095ED9A95F1F700008111CA
:1012D000F5CF8091E80085FF14C040E050E068E061
:1012E00070E0CE010E946A0B8091E8008E778093B7
:1012F000E80080E2FE01A2E9B1E001900D928A953A
:10130000E1F7DF91CF91089588EE92E00C944004CC
:10131000209190012F5F822F62E30E94211E99236A
:1013200019F02093900108951092900180919101FD
:10133000882371F180914902843041F58091E90060
:101340008F702091EC00922F917020FD90E8892BF6
:1013500093E09093E9009091EB0090FF14C090917E
:10136000EE0097FF10C09091E80095FF03C0109227
:10137000F100F9CF9091E80090FF05C09091E8004E
:101380009E779093E8008F708093E900109291010E
:10139000089542E061EC81E00E94750C42E061EC4E
:1013A00082E00E94750C42E261EC83E00E94750CC1
:1013B00042E261EC84E00C94750C80914B02833026
:1013C00009F455C030F4813071F0823009F48EC0D8
:1013D00008958A3009F47AC08B3009F460C08930EE
:1013E00009F09CC020C080914A02813A09F096C061
:1013F0008091E800877F8093E80080914E02909171
:101400004F02892B21F460E282E991E003C060E0A1
:1014100080E090E070E00E94B70B8091E8008B774D
:101420008093E800089580914A02813209F076C0E5
:1014300080914E0290914F02009719F0039709F0A6
:101440006DC08091E800877F8093E8008091E8007C
:1014500082FD05C0809149028111F8CF5FC0809163
:10146000F1008093B2018091E8008B7753C08091A6
:101470004A02813A09F052C080914E0290914F0287
:10148000892B09F04BC08091E800877F8093E800AA
:101490008091E80080FFFCCF80910B0136C08091E5
:1014A0004A028132D9F580914E0290914F02892BE8
:1014B000A9F58091E800877F8093E8000E94AA0C3C
:1014C00080914C0280930B010C94DC1480914A02B1
:1014D000813221F58091E800877F8093E8000E94A7
:1014E000AA0C80914D028093B301089580914A0225
:1014F000813AA1F48091E800877F8093E800809191
:10150000E80080FFFCCF8091B3018093F1008091CF
:10151000E8008E778093E8000C94AA0C0895089553
:101520000895089584EE92E00E9440040C94910A7C
:101530000E944A1B80914702882329F00E94751B54
:1015400081110C94540B089584B7877F84BF0FB624
:10155000F894A89580916000886180936000109253
:1015600060000FBE90E080E80FB6F89480936100B1
:10157000909361000FBE0E948F0A0E94FB0F0E9491
:10158000FB0C0E944E0D8091E20084608093E2008B
:1015900088E698E00E941F1B78948091490284306D
:1015A00019F00E94590FF9CF8FEC92E00E9440048D
:1015B0000E94FD0F81E091E00E94740F8EEB92E09B
:1015C0000E9440040E94900A80914902853039F4BB
:1015D0008AEB92E00E9440040E94980AF5CF0E9494
:1015E00001100E94590FF0CF0C94891B80EE92E0FD
:1015F0000E9440040C94F40A292F3327233031052C
:10160000C9F064F42130310581F02230310509F050
:1016100043C084E790E022E333E042C02132310549
:10162000F1F02232310541F137C082E190E026EA43
:1016300033E036C099278130910541F08230910521
:1016400041F0892B49F5EEE2F3E005C0EEE1F3E06D
:1016500002C0ECEEF2E0849190E09F0121C0643082
:10166000D8F4E62FF0E0EE0FFF1FE55EFE4F20817D
:10167000318189E090E014C0643070F470E0FB01C7
:10168000EE0FFF1FED5EFE4F20813181FB01E15F18
:10169000FE4F808190E004C080E090E020E030E0E8
:1016A000FA0131832083089584E089BD86E089BDF5
:1016B00009B400FEFDCF8091D8008F7D8093D800C3
:1016C0008091E00082608093E0008091E00081FDE5
:1016D000FCCF0895CF92DF92EF92FF920F931F936A
:1016E000CF93DF93EC018B017A010E94C90C811129
:1016F00035C0E114F10439F0F70180819181081BB4
:10170000190BC80FD91FC12CD12C0115110529F1B6
:101710008091E80085FD18C08091E8008E77809365
:10172000E8000E94590FE114F10449F0F7018081AB
:101730009181C80ED91ED182C08285E00FC00E945F
:10174000C90C882311F30AC089918093F1000150DC
:101750001109FFEFCF1ADF0AD8CF80E0DF91CF91D8
:101760001F910F91FF90EF90DF90CF9008952091FF
:101770005002309151022617370748F06115710564
:1017800039F42091E8002E772093E80001C0B901D8
:1017900040E06115710591F120914902222309F47D
:1017A00040C0253009F43FC02091E80023FD3DC032
:1017B0002091E80022FD2FC02091E80020FFE9CF12
:1017C0002091F20030E0FC01CF016115710559F064
:1017D0002830310540F481918093F1006150710906
:1017E0002F5F3F4FF1CF41E02830310509F040E055
:1017F0002091E8002E772093E800CBCF4111CCCF89
:101800000AC080914902882361F0853061F080919F
:10181000E80083FD0AC08091E80082FFF2CF80E0FB
:10182000089582E0089583E0089581E0089520916D
:101830005002309151022617370748F061157105A3
:1018400039F42091E8002E772093E80001C0B90117
:10185000FC0120E06115710579F18091490288232E
:1018600009F43DC0853009F43CC08091E80083FD57
:101870003AC08091E80082FD2CC08091E80080FF92
:10188000E9CF8091F20090E06115710559F0883040
:10189000910540F424912093F10031966150710933
:1018A0000196F2CF21E0089709F020E08091E8004E
:1018B0008E778093E800CECF2111CFCF0AC08091E0
:1018C0004902882361F0853061F08091E80083FD52
:1018D0000AC08091E80082FFF2CF80E0089582E0A4
:1018E000089583E0089581E00895982F953058F584
:1018F0009093E900981739F07091EC002091ED0079
:101900005091F00003C0242F762F50E021FF19C022
:101910003091EB003E7F3093EB003091ED003D7F46
:101920003093ED003091EB0031603093EB00709319
:10193000EC002093ED005093F0002091EE0027FF83
:1019400007C09F5FD3CF8F708093E90081E0089537
:1019500080E0089580914A0287FF11C08091E800DD
:1019600082FD05C0809149028111F8CF11C080919C
:10197000E8008B770BC080914902882349F0809161
:10198000E80080FFF8CF8091E8008E778093E80030
:1019900008952091E4003091E50095E64091EC0037
:1019A000842F817040FF22C08091E80080FD1CC020
:1019B00080914902882391F0853091F08091EB006D
:1019C00085FD10C04091E4005091E5004217530797
:1019D00029F39A01915011F784E0089582E0089567
:1019E00083E0089581E0089580E008954091E80043
:1019F00042FFDECF08950E94580D0E945B0DE0EE7D
:101A0000F0E0808181608083E8EDF0E080818F7775
:101A1000808319BCE3E6F0E08081816080831092CE
:101A2000480208950E94580D0E945B0D8091D800D5
:101A30008F778093D8008091D80080688093D800F9
:101A40008091D8008F7D8093D80084E089BD86E0A6
:101A500089BD09B400FEFDCF1092490210924502E3
:101A6000109247021092460242E060E080E00E943D
:101A7000750C8091E1008E7F8093E1008091E200FF
:101A800081608093E2008091E20088608093E200B0
:101A90008091E0008E7F8093E0000895E3E6F0E01F
:101AA00080818E7F808381E0809348020C94120DA8
:101AB0001092E20008951092E10008951F920F9293
:101AC0000FB60F9211242F933F934F935F936F9311
:101AD0007F938F939F93AF93BF93EF93FF938091E7
:101AE000E10082FF0BC08091E20082FF07C080917D
:101AF000E1008B7F8093E1000E9488098091E100E2
:101B000080FF19C08091E20080FF15C08091E20043
:101B10008E7F8093E2008091E20080618093E200FA
:101B20008091D80080628093D80019BC85E08093B2
:101B300049020E94920A8091E10084FF30C08091A6
:101B4000E20084FF2CC084E089BD86E089BD09B431
:101B500000FEFDCF8091D8008F7D8093D8008091CA
:101B6000E1008F7E8093E1008091E2008F7E809380
:101B7000E2008091E20081608093E2008091450262
:101B8000882311F084E007C08091E30087FD02C044
:101B900081E001C083E0809349020E94F60A8091AF
:101BA000E10083FF24C08091E20083FF20C0809188
:101BB000E100877F8093E10082E0809349021092E8
:101BC00045028091E1008E7F8093E1008091E200E8
:101BD0008E7F8093E2008091E20080618093E2003A
:101BE00042E060E080E00E94750C0E948409FF9151
:101BF000EF91BF91AF919F918F917F916F915F9185
:101C00004F913F912F910F900FBE0F901F901895FD
:101C10001F93CF93DF93CDB7DEB7AA970FB6F89493
:101C2000DEBF0FBECDBFEAE4F2E088E08E0F9091F8
:101C3000F10091938E13FBCF0E94DD098091E800A3
:101C400083FF1FC180914A0290914B02492F50E0BF
:101C50004A30510508F015C1FA01E85BFF4F0C94BA
:101C60002D1E803881F0823809F00BC180914E0220
:101C70008F708093E9008091EB0085FB882780F9C5
:101C80001092E90006C0809146029091470291119E
:101C900082609091E800977F9093E8008093F10034
:101CA0001092F100C8C0282F2D7F09F0EAC08823C8
:101CB00019F0823061F0E5C080914C02813009F06A
:101CC000E0C0933009F080E0809347022BC0809100
:101CD0004C02811127C080914E028F7009F4D1C04F
:101CE0008093E9002091EB0020FF1CC0933021F489
:101CF0008091EB00806214C09091EB009061909312
:101D0000EB0021E030E0A90102C0440F551F8A9585
:101D1000E2F74093EA001092EA008091EB008860BD
:101D20008093EB001092E9008091E800877F86C0E5
:101D30008111A7C010914C021F778091E300807839
:101D4000812B8093E3008091E800877F8093E800F7
:101D50000E94AA0C8091E80080FFFCCF8091E300F4
:101D600080688093E300111102C082E001C083E02B
:101D70008093490286C08058823008F082C08091EA
:101D80004C0290914D028C3D53E0950779F583E02C
:101D90008A838AE289834FB7F894DE01139620E0A4
:101DA0003EE051E2E32FF0E050935700E49120FF32
:101DB00003C0E295EF703F5FEF708E2F90E0EA3046
:101DC00010F0C79601C0C0968D939D932F5F24316C
:101DD00049F74FBF8091E800877F8093E8006AE26F
:101DE00070E0CE0101960E94B70B14C0AE014F5FA8
:101DF0005F4F60914E020E94FC0ABC01892B09F4DE
:101E000040C09091E800977F9093E80089819A8183
:101E10000E94170C8091E8008B778093E80031C016
:101E2000803879F58091E800877F8093E800809181
:101E300045028093F1008091E8008E778093E8005E
:101E40000E94AA0C1EC081111CC090914C029230BD
:101E5000C0F48091E800877F8093E800909345026A
:101E60000E94AA0C80914502811106C08091E30076
:101E700087FD02C081E001C084E0809349020E9496
:101E8000C9098091E80083FF0AC08091E800877F3C
:101E90008093E8008091EB0080628093EB00AA962B
:101EA0000FB6F894DEBF0FBECDBFDF91CF911F916B
:101EB0000895CF93809149028823A1F0C091E90051
:101EC000CF709091EC00892F817090FD80E8C82B35
:101ED0001092E9008091E80083FD0E94080ECF7007
:101EE000C093E900CF9108959093B9018093B80110
:101EF0000895E091B801F091B901309721F0019077
:101F0000F081E02D099480E00895EF92FF920F9305
:101F10001F93CF93DF93E091B801F091B90130970F
:101F2000B1F18C010280F381E02D099580913E0290
:101F300082FF2DC080FF04C081E994E00E9440042C
:101F4000E80110E28BE8E82E84E0F82E80913E0252
:101F500080FF0BC088811F928F93FF92EF920E94A7
:101F6000D9040F900F900F900F90115021961111DE
:101F7000EDCF80913E0280FF0AC089E894E0DF91B6
:101F8000CF911F910F91FF90EF900C944004DF913F
:101F9000CF911F910F91FF90EF9008952091B6017E
:101FA0003091B7018217930771F09093B701809336
:101FB000B601E091B801F091B901309721F00680A7
:101FC000F781E02D099408952091B4013091B50175
:101FD0008217930771F09093B5018093B401E0915B
:101FE000B801F091B901309721F00084F185E02D1E
:101FF0000994089508950C94FA0F0E94B41B0C9450
:102000002505CF92DF92EF92FF920F931F93CF930C
:10201000DF9300D000D000D0CDB7DEB70E943405EA
:102020008BEBC82E81E0D82E00E010E0E02E802F50
:102030000E941A06F60141916F01F42EF826B1F4C0
:102040000F5F1F4F0032110589F78FEF89838A8355
:102050001B820E94BD1B8160782F9D838C834981E8
:102060005A816B818D810E94BE1047C090913E02C3
:1020700091FF04C08E830E9420068E8120E030E014
:102080004F2D50E0922FBA01022E02C07595679530
:102090000A94E2F760FF2BC02983EA8221E030E056
:1020A000690102C0CC0CDD1C9A95E2F790E08C210E
:1020B0009D21892B09F420E02B830E94BD1B8160A8
:1020C000782F9D838C8349815A816B818D810E94F9
:1020D000BE1049815A816B817C818D810E94371BA2
:1020E000F801E554FE4F8081C826C08206C02F5FEC
:1020F0003F4F2830310531F6A3CF0E94361B109197
:10210000BA010E94790F181741F10E94790F80934C
:10211000BA0190913E0292FF0EC090FF0CC01F9238
:102120008F9383EA94E09F938F930E94D9040F903A
:102130000F900F900F908091BA0126960FB6F894E9
:10214000DEBF0FBECDBFDF91CF911F910F91FF90EA
:10215000EF90DF90CF900C94481B26960FB6F89422
:10216000DEBF0FBECDBFDF91CF911F910F91FF90CA
:10217000EF90DF90CF9008950C946606CF93DF9395
:10218000CDB7DEB72B970FB6F894DEBF0FBECDBF2D
:10219000942F4F83252F588769877A878B874A85A5
:1021A0005B85452B21F02F3F09F59F3FF9F4DE01B8
:1021B000119686E0FD0111928A95E9F785E0FE010E
:1021C000379601900D928A95E1F749815A816B818A
:1021D0007C818D819E810E9485172B960FB6F89485
:1021E000DEBF0FBECDBFDF91CF9108954F815885DF
:1021F00069857A858B850E94371BD9CFCF93882339
:1022000009F4A4C0C82F8CEF8C0F813A48F48C2FAE
:102210000E94C11D81119AC08C2F0E94141A0CC0FB
:1022200080E28C0F883058F4C77081E001C0880FBD
:10223000CA95EAF70E94BF1ACF910C94F91A8BE560
:102240008C0F833078F4C53A29F0C63A31F083E830
:1022500090E005C081E890E002C082E890E0CF9174
:102260000C94CE0F88E58C0F853108F06FC0C83A0A
:1022700061F1C93A69F1CA3A71F1CB3A79F1CC3AD4
:1022800081F1CD3A89F1CE3A91F1CF3A99F1C13B42
:10229000A1F1C03BA9F1C23BB1F1C33BB9F1C43BD1
:1022A000C1F1C53BC9F1C63BD1F1C73BD9F1C83B30
:1022B000E1F1C93BE9F1CA3BF1F1CB3BF9F1CC3B90
:1022C00009F43FC080E090E03EC082EE90E03BC069
:1022D00089EE90E038C08AEE90E035C085EB90E062
:1022E00032C086EB90E02FC083EB90E02CC084EBF3
:1022F00090E029C087EB90E026C08CEC90E023C0F2
:102300008DEC90E020C083E891E01DC08AE891E068
:102310001AC082E991E017C084E991E014C081E21B
:1023200092E011C083E292E00EC084E292E00BC022
:1023300085E292E008C086E292E005C087E292E082
:1023400002C08AE292E0CF910C94E40FCF910895FD
:10235000882329F19CEF980F913A18F40E94671A8C
:102360000DC090E2980F983058F4877091E001C04A
:10237000990F8A95EAF7892F0E94C51A0C94F91AC9
:102380009BE5980F933020F480E090E00C94CE0F02
:10239000885A853120F480E090E00C94E40F089591
:1023A000882321F00E94BF1A0C94F91A08958823FB
:1023B00021F00E94C51A0C94F91A0895CF92DF9269
:1023C000EF92FF920F931F93CF93DF9300D000D033
:1023D00000D0CDB7DEB725E0FC01DE0111960190FB
:1023E0000D922A95E1F7FC0140813181F28025812F
:1023F00022952F7063817481672B09F4C0C23F3F1F
:1024000019F44F3F09F4BBC26C0149833A838981B7
:102410009A812E830E94D319182F092F0E94D21956
:102420000E94E218E02FE295EF70F0E0EE5AFF4FC5
:102430002E810C942D1E802F807F902F9F70092F4E
:10244000882311F00295007FFF2049F0002309F452
:1024500047C2802F0E94D21A0E94F91A41C2812FCE
:102460000E94A811002309F48AC2802F0E94D81A62
:1024700026960FB6F894DEBF0FBECDBFDF91CF9189
:102480001F910F91FF90EF90DF90CF900C94F91A6D
:10249000802F807F902F9F70092F803211F002953E
:1024A000007F112319F0113001F129C0FF20A9F09C
:1024B000802F222349F1213039F526960FB6F89462
:1024C000DEBF0FBECDBFDF91CF911F910F91FF9067
:1024D000EF90DF90CF900C94E21A222319F0213074
:1024E00009F44DC20E94E51A2CC0FF20E9F0263005
:1024F00008F045C20E94BC1A802329F022C0FF20A8
:10250000F1F0211115C0802F26960FB6F894DEBF8A
:102510000FBECDBFDF91CF911F910F91FF90EF9034
:10252000DF90CF900C94D011253008F028C209C05C
:10253000F601858180FFD4C18F708583E4CF21119E
:10254000E3C1802F51C1202F26952695237030E0BE
:102550002115310521F021303105C9F010C2FF20CD
:1025600021F0812F902F937002C080E090E026969A
:102570000FB6F894DEBF0FBECDBFDF91CF911F9194
:102580000F91FF90EF90DF90CF900C94CE0FFF2033
:1025900021F0812F902F937002C080E090E026966A
:1025A0000FB6F894DEBF0FBECDBFDF91CF911F9164
:1025B0000F91FF90EF90DF90CF900C94E40F802F5D
:1025C000837009F078C0F110DAC1812F8295869569
:1025D0008770880F880F912F9F70C92ED12CE12C06
:1025E000F12C082E04C0CC0CDD1CEE1CFF1C0A9440
:1025F000D2F714FF12C04FE050E060E070E004C07A
:10260000440F551F661F771F8A95D2F7CB01BA0179
:10261000609570958095909503C060E070E0CB0167
:10262000202F269526952370422F50E042305105E9
:10263000D1F04330510559F16C297D298E299F290C
:102640004130510541F126960FB6F894DEBF0FBE1A
:10265000CDBFDF91CF911F910F91FF90EF90DF9051
:10266000CF900C94F7186C297D298E299F292696E6
:102670000FB6F894DEBF0FBECDBFDF91CF911F9193
:102680000F91FF90EF90DF90CF900C9409190E946A
:10269000F718C701B60126960FB6F894DEBF0FBE35
:1026A000CDBFDF91CF911F910F91FF90EF90DF9001
:1026B000CF900C94E518FF2019F0802F817001C095
:1026C0008695882309F45BC1812F82958695877052
:1026D000880F880F912F9F70C92ED12CE12CF12CDF
:1026E000082E04C0CC0CDD1CEE1CFF1C0A94D2F793
:1026F00014FF12C04FE050E060E070E004C0440FEF
:10270000551F661F771F8A95D2F7CB01BA016095D6
:1027100070958095909503C060E070E0CB01202F0C
:10272000269526952370422F50E042305105D1F076
:102730004330510559F16C297D298E299F2941305B
:10274000510541F126960FB6F894DEBF0FBECDBFFE
:10275000DF91CF911F910F91FF90EF90DF90CF907D
:102760000C94AE196C297D298E299F2926960FB6C7
:10277000F894DEBF0FBECDBFDF91CF911F910F91B7
:10278000FF90EF90DF90CF900C94C0190E94AE198B
:10279000C701B60126960FB6F894DEBF0FBECDBFB7
:1027A000DF91CF911F910F91FF90EF90DF90CF902D
:1027B0000C949C19103F41F118F4103E48F48BC062
:1027C000123F09F450C0D8F1133F09F460C083C030
:1027D0001F70802F8F71FF2021F00E943519812FEB
:1027E00093CE0E945619812F26960FB6F894DEBF1D
:1027F0000FBECDBFDF91CF911F910F91FF90EF9052
:10280000DF90CF900C94D711FF20A9F0253008F06D
:10281000B6C0802F8F7126960FB6F894DEBF0FBE1C
:10282000CDBFDF91CF911F910F91FF90EF90DF907F
:10283000CF900C947B19263008F0A1C0EACFFF207E
:10284000A1F0802F8F7126960FB6F894DEBF0FBED1
:10285000CDBFDF91CF911F910F91FF90EF90DF904F
:10286000CF900C943519FF2061F3802F8F7126963D
:102870000FB6F894DEBF0FBECDBFDF91CF911F9191
:102880000F91FF90EF90DF90CF900C945619FF209E
:1028900091F0802F8F7126960FB6F894DEBF0FBE91
:1028A000CDBFDF91CF911F910F91FF90EF90DF90FF
:1028B000CF900C94201926960FB6F894DEBF0FBE69
:1028C000CDBFDF91CF911F910F91FF90EF90DF90DF
:1028D000CF900C941B19FF20A1F0222309F4B1CF53
:1028E000812F26960FB6F894DEBF0FBECDBFDF91C5
:1028F000CF911F910F91FF90EF90DF90CF900C94AC
:10290000FE10222309F4B1CF812F26960FB6F8943A
:10291000DEBF0FBECDBFDF91CF911F910F91FF9012
:10292000EF90DF90CF900C94A811402F4F70612F43
:10293000C6010E945C1C26960FB6F894DEBF0FBE3F
:10294000CDBFDF91CF911F910F91FF90EF90DF905E
:10295000CF900C942D18402F4F70612FC6012696F2
:102960000FB6F894DEBF0FBECDBFDF91CF911F91A0
:102970000F91FF90EF90DF90CF900C945F1C269604
:102980000FB6F894DEBF0FBECDBFDF91CF911F9180
:102990000F91FF90EF90DF90CF9008950E94DF1A83
:1029A0000E94AE1A0E94F91A80E090E00E94CE0FB9
:1029B00080E090E00C94E40F0E94CF1A0C94CE14A7
:1029C0000E94D319292F22952F7030E02C30310529
:1029D0004CF42A3031056CF4225031092230310593
:1029E00088F407C02C30310549F02F30310531F023
:1029F00009C0803E48F0803F29F406C093FB882739
:102A000080F9089580E0089581E00895CF93DF93E1
:102A100000D000D01F92CDB7DEB70F900F900F906F
:102A20000F900F90DF91CF910895CF93DF9300D057
:102A300000D000D0CDB7DEB726960FB6F894DEBF33
:102A40000FBECDBFDF91CF910895CF93DF93C0919B
:102A5000DB018091DC01C817A1F0D0E0CE0166E077
:102A600070E00E94101EFC01E352FE4F4081518134
:102A700062817381848195810E9415152196C770AA
:102A8000E8CFDF91CF91089540910D0250910E0251
:102A900060910F02709110028091110290911202C8
:102AA0000C941515CF93DF938091120282958F704D
:102AB00009F05CC080910F02882309F457C020916F
:102AC000DB01D091DC0140910D02C0910E02E0913A
:102AD0001002F09111022D1709F448C030E0309730
:102AE00009F440C0CF3F11F44F3FE1F1C90166E066
:102AF00070E00E94101EDC01A352BE4F11968C9113
:102B00001197C8132FC08C9148132CC012968C912A
:102B10001297811127C013968D919C9114978E174F
:102B20009F0708F401978E1B9F0B883C9105D0F4FA
:102B3000809112028F70806180931202C90166E059
:102B400070E00E94101EFC01EE51FE4F90819F70BC
:102B5000906190838DE092E00E94DE11DF91CF9131
:102B60000C9425152F5F3F4F2770B5CFDF91CF9184
:102B70000895BF92CF92DF92EF92FF920F931F932F
:102B8000CF93DF93CDB7DEB761970FB6F894DEBF72
:102B90000FBECDBF8C0185E0F801DE011D960190CE
:102BA0000D928A95E1F7D8014C9111962C911197CD
:102BB0001296EC9012971396CD90DC90149750914A
:102BC0000D0260910E028091100290911102009707
:102BD00009F46EC16F3F19F45F3F09F469C1B09009
:102BE0000F02BB2009F4C3C030911202C816D906E7
:102BF00028F0F601E81BF90BCF0104C080959095F1
:102C00008C0D9D1DFF24F394883C910588F0F12CD8
:102C1000307F09F0CBC07C2DD98AC88A522F6E2D07
:102C200089890E9406158DE092E00E94DE11B4C0F1
:102C3000832F807F09F049C0621314C0541312C05F
:102C4000E11010C03F703061309312020E944415B1
:102C50008DE092E00E94DE1180911202D80115965B
:102C60008C9331C0CD2831F12F3F11F44F3F11F13A
:102C7000FE2CE1101FC0E091DB013091DC01E31775
:102C800009F45CC0F0E0CF0166E070E00E94101E25
:102C9000DC01A352BE4F11968C911197281307C0E7
:102CA0008C91481304C012968C91811103C0319607
:102CB000E770E5CFFE2CEE2009F416C180911202D8
:102CC000816080931202F12C0FC1621308C054136B
:102CD00006C0E11004C080911202D801C1C04D8726
:102CE0002E878D859E850E94E0148823E1F1EE20D9
:102CF000D1F120911202822F82958F7090E002977D
:102D000074F080910D0290910E0298878F8319863E
:102D1000DB86CA862C87CE0107960E94DE1186E0EC
:102D2000F801ADE0B2E001900D928A95E1F70E94C2
:102D300052150E944415FF24F394D6C04D872E8768
:102D40008D859E850E94D319292F22952F7030E002
:102D5000223031050CF0BCC09F7009F0B6C0805E17
:102D6000883008F4C1C0C8010E94DE11E4CFC81643
:102D7000D90608F453C0F601E81BF90BCF01883CD3
:102D8000910508F450C0F12C7C2DD98AC88A522FA5
:102D90006E2D89890E940615EDE0F2E086E0DF01E4
:102DA0001D928A95E9F70E9444159EC0621314C0D3
:102DB000541312C0E11010C080911202F8018583F3
:102DC000C8010E94DE1186E0EDE0F2E0DF011D9215
:102DD0008A95E9F7FB2C88C04D872E878D859E85C7
:102DE0000E94E014882309F4BECFEE2009F4BBCF83
:102DF00020911202822F82958F7090E002970CF43E
:102E00008ECF80910D0290910E029A8389831B824E
:102E1000DD82CC822E83CE0101967FCF8095909566
:102E20008C0D9D1DACCFFE2CEE2009F49CCF6213BF
:102E30002EC054132CC02091120220FD1FC0822FDF
:102E400082958F70D9F0D80115962C9315978F30F5
:102E500049F08F5F982F9295907F822F8F70892BEA
:102E600015968C93C8010E94DE1186E0F801ADE052
:102E7000B2E001900D928A95E1F795CF86E0F801D6
:102E8000ADE0B2E001900D928A95E1F72DC04D873B
:102E90002E878D859E850E94E014811140CF809100
:102EA0001202816080931202C8010E94DE111CC0D0
:102EB000EE2009F458CF4D872E878D859E850E9480
:102EC000E014882309F44FCF2ACF811148CF0CC0DA
:102ED000243031050CF047CF9F7009F440CFF80142
:102EE0009581907F09F03BCF8F2D61960FB6F894B6
:102EF000DEBF0FBECDBFDF91CF911F910F91FF902D
:102F0000EF90DF90CF90BF900895CF93DF93CDB730
:102F1000DEB72C970FB6F894DEBF0FBECDBF4F8340
:102F2000588769877A878B879C87CE0107960E948E
:102F3000B915882371F08F8198852A853B85232BCD
:102F400009F43FC09F3F09F068C08F3F09F065C09A
:102F500038C086E0FE013796DE01119601900D9291
:102F60008A95E1F76F817885EA85FB85309749F18D
:102F70007F3F11F46F3F29F18091DC0190E09C01CB
:102F80002F5F3F4F277033274091DB0150E024171C
:102F9000350709F44BC069837A83FD83EC8366E0CF
:102FA00070E00E94101EDC01A352BE4F96E0FE01AD
:102FB000319601900D929A95E1F72093DC010E94E1
:102FC00025158091DB019091DC018917E9F190E0F2
:102FD00066E070E00E94101E83529E4F0E94B91559
:102FE000882391F18091DB0190E066E070E00E941F
:102FF000101EFC01E352FE4F4081518162817381BA
:10300000848195810E9415158091DB0190E00196E5
:10301000877099278093DB01D4CF4F8158856985CC
:103020007A858B859C850E941515CBCF0E94DC1478
:103030001092DC011092DB01EDE0F2E086E0DF01AE
:103040001D928A95E9F7BDCF2C960FB6F894DEBF96
:103050000FBECDBFDF91CF910895DF92EF92FF9227
:103060000F931F93CF93DF93FC01892B09F48AC040
:10307000E12CF12CDD24D394EF0121968491853746
:1030800009F461C058F4843708F04EC0843008F069
:103090006AC08130D1F0823071F174C0883709F490
:1030A0005DC050F4863709F455C0873709F06AC00F
:1030B0008E2D0E94CC1A54C09CE7980F903708F0D0
:1030C00061C08F770E94A81150C08F010E5F1F4F03
:1030D000FE01849190E2980F983050F48770FD2D96
:1030E00001C0FF0F8A95EAF78F2F0E94D21A14C0F1
:1030F0000E94FE1013C08F010E5F1F4FFE01C4918E
:1031000080E28C0F883060F4C7708D2D01C0880F6D
:10311000CA95EAF70E94D81A0E94F91AE80125C058
:103120008C2F0E94A811FACF9F012E5F3F4FFE0106
:10313000C491CC2369F08FE99FE00197F1F700C0BB
:103140000000C150F6CF9F012E5F3F4FFE01F4906B
:10315000E9010BC00E94BC1AE82E07C00E94CF1ADA
:103160000E94F91A02C00E94FE108F2D882341F0A0
:10317000EFE9FFE03197F1F700C000008150F6CF92
:10318000FE017ACFDF91CF911F910F91FF90EF90C9
:10319000DF900895609317027093180280931902CC
:1031A00090931A020E94461B0C94CE146093130253
:1031B0007093140280931502909316020E94471B8D
:1031C0000C94CE1408950C94CA180F931F93009179
:1031D0001702109118022091190230911A02602BE7
:1031E000712B822B932B1F910F910C94CA180F9364
:1031F0001F9300911702109118022091190230912B
:103200001A0260237123822393231F910F910C9440
:10321000CA180F931F930091170210911802209162
:10322000190230911A0260277127822793271F9174
:103230000F910C94CA1860E070E0CB010C94D61882
:103240000F931F9341E050E060E070E08A019B0122
:1032500004C0000F111F221F331F8A95D2F7C90126
:10326000B8011F910F910C94D6180F931F9341E052
:1032700050E060E070E004C0440F551F661F771FE8
:103280008A95D2F78091130290911402A0911502B1
:10329000B09116028A019B01082B192B2A2B3B2B7C
:1032A000C901B8011F910F910C94D6180F931F9369
:1032B00041E050E060E070E004C0440F551F661F1D
:1032C000771F8A95D2F740955095609570958091BB
:1032D000130290911402A0911502B09116028A0176
:1032E0009B01082319232A233B23C901B8011F91FD
:1032F0000F910C94D6180F931F9341E050E060E0BB
:1033000070E004C0440F551F661F771F8A95D2F7DF
:103310008091130290911402A0911502B0911602AF
:103320008A019B01082719272A273B27C901B801D1
:103330001F910F910C94D6180F931F9300911302B5
:10334000109114022091150230911602602B712BFE
:10335000822B932B1F910F910C94D6180F931F93D0
:10336000009113021091140220911502309116025F
:1033700060237123822393231F910F910C94D618FD
:103380000F931F93009113021091140220911502C4
:103390003091160260277127822793271F910F9182
:1033A0000C94D6180895CF92DF92EF92FF920F936C
:1033B0001F93CF93DF938C01C0901702D090180217
:1033C000E0901902F0901A024091130250911402F9
:1033D0006091150270911602C42AD52AE62AF72AAE
:1033E000CFE1D0E0D701C6010C2E04C0B695A79559
:1033F000979587950A94D2F780FF07C0B8018C2F64
:103400000E942D1C8130910531F4219758F7B801A5
:1034100080E00E942D1CDF91CF911F910F91FF90B2
:10342000EF90DF90CF90089590910B01992321F0B8
:1034300090910C01911109C020910D0130910E0164
:10344000F90132969FEF40E030C0982F96959695FF
:1034500096959F31A0F4E0910D01F0910E01E90FD6
:10346000F11D877021E030E0A90102C0440F551F13
:103470008A95E2F7CA019181892B81830895909101
:103480003E0290FF23C01F928F938CEC94E09F9399
:103490008F930E94D9040F900F900F900F90089572
:1034A0009F3F39F04F5F4E3141F051915813F8CFA3
:1034B0000DC05111F7CF942FF5CF9F3F39F0F9018F
:1034C000E90FF11D97FDFA95828308950895909173
:1034D0000B01992321F090910C01911109C02091C9
:1034E0000D0130910E01F9013296205E3F4F30C040
:1034F000982F9695969596959F31A8F4E0910D0199
:10350000F0910E01E90FF11D877021E030E0A90173
:1035100002C0440F551F8A95E2F7CA018095918138
:1035200089238183089590913E0290FF16C01F92D7
:103530008F938EEA94E09F938F930E94D9040F900B
:103540000F900F900F9008953196E217F30729F02E
:1035500090819813F9CF1082F7CF089581E090E021
:10356000E0910D01F0910E01E80FF91F1082019614
:1035700080329105A9F7089580913D0208959091B8
:103580003D02892B80933D020895809590913D02E4
:10359000892380933D02089580933D0208951092FF
:1035A0003D02089590913C02892B80933C0208953E
:1035B000809590913C02892380933C02089510925B
:1035C0003C02089580931B02089510921B020895F7
:1035D00080910D0190910E01FC0131969C01205EBD
:1035E0003F4F80E0919191118F5FE217F307D1F780
:1035F0000895E0910D01F0910E0180913D028083CC
:10360000E0910D01F0910E01908180913C02892B97
:10361000808380911B02882361F0E0910D01F0917D
:103620000E019081892B80830E94E81A81111092EB
:103630001B0280910D0190910E010C94850F9093C7
:1036400025018093240108958295982F9C7C292F31
:1036500026952695982F9373990F990F922B892F62
:103660008A7A86959575990F892B08950895CF9339
:10367000DF9300D000D01F92CDB7DEB70F900F9030
:103680000F900F900F90DF91CF91089508950895B6
:103690000C94BC1080914902843021F110923F02B9
:1036A00020E488E190E00FB6F894A895809360003C
:1036B0000FBE2093600083B7817F846083BF83B790
:1036C000816083BF7894889583B78E7F83BF0FB660
:1036D000F894A895809160008861809360001092B2
:1036E00060000FBE089508950895CF930E94731B44
:1036F0000E9434050E94741BC0E08C2F0E941A06A1
:10370000811104C0CF5FC032C1F701C081E0CF9109
:1037100008950C94DC141F920F920FB60F9211248F
:103720008F939F93AF93BF9380913F02811113C0FA
:103730008091400290914102A0914202B0914302D7
:103740004196A11DB11D8093400290934102A09328
:103750004202B0934302BF91AF919F918F910F901E
:103760000FBE0F901F90189582E084BD93E095BD29
:103770009AEF97BD80936E0008952FB7F8948091CB
:10378000400290914102A0914202B09143022FBFAA
:1037900008952FB7F8946091400270914102809192
:1037A0004202909143022FBF08951F920F920FB6CD
:1037B0000F9211248F939F93AF93BF9380914002F8
:1037C00090914102A0914202B09143020196A11D45
:1037D000B11D8093400290934102A0934202B093A6
:1037E0004302BF91AF919F918F910F900FBE0F90A9
:1037F0001F9018950E94FB0CF8942FEF87EA91E632
:10380000215080409040E1F700C0000087E090EB3D
:10381000DC018093520290935302A0935402B09320
:1038200055029CE088E10FB6F894A895809360005B
:103830000FBE90936000FFCFE92FF0E093E0EE0F12
:10384000FF1F9A95E1F7E80FF11DEC53FF4F94919C
:10385000892F8F7092959F700895CF93C82FCB01B9
:103860000E941C1C492F90E0242F30E054E0220FCE
:10387000331F5A95E1F7282B392B2038310519F4DD
:1038800080E090E017C0EC2FF0E023E0EE0FFF1F88
:103890002A95E1F74770E40FF11D34E0EE0FFF1FAA
:1038A0003A95E1F7E80FF91FEE0FFF1FE050F849D6
:1038B00085919491CF91089580E090E008950895C6
:1038C000CF93C82F1F928F9380EF94E09F938F9395
:1038D0000E94D90481E090E0A0E0B0E0BC01CD01FD
:1038E00004C0660F771F881F991FCA95D2F70E94E0
:1038F000E3180F900F900F900F90CF910C94DC1461
:10390000CF938732A8F58E3108F02BC1803109F4AE
:103910009FC0F8F4873009F464C0A8F4863009F039
:1039200024C180913E02817F8E7F80933E0285EF8D
:1039300094E00E94400481ED97E00E94400481E001
:10394000809344024CC08B30F1F18E3009F46CC08E
:103950000CC1863109F4B0C020F4813109F4EDC006
:1039600004C1893109F491C08B3109F449C0FDC00B
:10397000883349F150F4893209F4F1C0853309F4F0
:10398000EEC0873209F0F1C0EAC0833409F4E7C021
:1039900028F48A3308F4E9C08953E4C0883409F074
:1039A000E4C00E94DC1480EC97E00E9440042FEFFA
:1039B00083ED90E3215080409040E1F700C000008B
:1039C0000E94FA1B0CC080E195E05CC087EA97E09A
:1039D0000E94400480913E02816080933E02C1E0DB
:1039E000C9C080913E02C82FC17080FFEFCF83EB2A
:1039F00097E00E94400480913E02817F8E7F3DC00F
:103A000090913E0291FBCC27C0F981E0C827892F15
:103A1000C0FB81F980933E02CC2319F08AE997E03C
:103A200027C08CE897E02EC090913E0292FBCC27F5
:103A3000C0F981E0C827892FC0FB82F980933E023C
:103A4000CC2319F08DE797E013C08DE697E01AC0FC
:103A500090913E0293FBCC27C0F981E0C827892FC3
:103A6000C0FB83F980933E02CC2351F081E697E0BE
:103A70000E94400480913E02816080933E027AC0A1
:103A800084E597E00E944004AACF85E497E00E9475
:103A9000400481E297E00E9440048BED96E00E9492
:103AA00040048EEA96E00E9440048DE696E00E9473
:103AB00040048EE396E0E6CF80E396E00E94400467
:103AC0000E94790F1F928F9386E196E09F938F93C8
:103AD0000E94D90480910B011F928F938FEF95E084
:103AE0009F938F930E94D9048091B3011F928F936B
:103AF0008CEE95E09F938F930E94D90480910C01E6
:103B00001F928F9389ED95E09F938F930E94D90424
:103B10000E94C91B9F938F937F936F9382EC95E0D4
:103B20009F938F930E94D9048DB79EB746960FB688
:103B3000F8949EBF0FBE8DBF52CF0E94DC14C0917F
:103B40000C0181E0C827C0930C01CC2329F088EB3D
:103B500095E00E9440040EC08DEA95E093CF80E08E
:103B600001C08D510E94601C3ACF8BEA95E00E9403
:103B70004004C0E08C2FCF91089580E0089580E04C
:103B80000895CF93C82F80914402882319F0813083
:103B900049F03EC0E0910D01F0910E01808182322A
:103BA000C9F507C0E0910D01F0910E0180818232CC
:103BB00061F48C2F0E94BD1D811104C08C2F0E94C6
:103BC000801C24C081E090E021C08C2F0E94BF1D8A
:103BD00081111BC0C43189F018F4CB3029F010C01A
:103BE000C93259F0C83361F485EF94E00E94400473
:103BF0008CEE94E00E94400408C0109244020CC075
:103C00008AEE94E00E94400407C081E0817006C003
:103C10001092440280E002C080E0F8CFCF91089576
:103C20000024552704C0080E591F880F991F0097BC
:103C300029F076956795B8F37105B9F7802D952F22
:103C40000895991B79E004C0991F961708F0961BF8
:103C5000881F7A95C9F780950895EE0FFF1F05908C
:0A3C6000F491E02D0994F894FFCFD1
:103C6A0001640833096708FF08CB0801011C0240F8
:103C7A0036223949041304F103B80344035D037679
:043C8A00039603009A
:106800008800EA44E944E244040005000600070069
:10681000080009000A000B000C000D000E000F001C
:1068200010001100120013001400150016001700CC
:10683000180019001A001B001C001D001E001F007C
:10684000200021002200230024002500260027002C
:10685000280029002A002B002C002D002E002F00DC
:1068600030003100000033003400350036003700BE
:10687000380039003A003B003C003D003E003F003C
:1068800040004100420043004400450046004700EC
:10689000480049004A004B004C004D004E004F009C
:1068A000500051005200530054005500560057004C
:1068B000580059005A005B005C005D005E005F00FC
:1068C00060006100620063006400F1A18500670060
:1068D000680069006A006B006C006D006E006F005C
:1068E0007000710072007300890087008A008B00BD
:1068F000E000E100E200E300E400E500E600E7007C
:106900000100010001000100EA4401000100E2442D
:106910000100010001000100460001004A004B0097
:10692000010001004700480001000100E9440100A6
:106930000100010001000100010001003A003B00DC
:106940003C003D003E003F0040004100420043004B
:10695000010035004C0001000100440045005200D8
:1069600049000100010050004F0029004D004E0079
:1069700051000100010001000100010001000100BF
:1069800001000100010001000100010001000100FF
:1069900001000100010001000100010001004D00A3
:1069A0004A004E004B0001000100010001000100FF
:1069B00001000100010001000100010001000100CF
:1069C00001000100010001000100010001000100BF
:1069D00001000100010001000100010001000100AF
:1069E0000100010001000100490001000100010057
:1069F000010001000100010001000100010001008F
:00000001FF
